:100000000C94AE130C94D8130C94D8130C94D813EE
:100010000C94D8130C94D8130C94D8130C94D813B4
:100020000C94D8130C94D8130C941CE70C9499E7F7
:100030000C94D8130C94D8130C94D8130C94D81394
:100040000C94D8130C94DC940C94D8130C94D813FF
:100050000C94D8130C94D8130C949EAA0C947BE6A1
:100060000C94D8130C94D8130C94D8130C94D81364
:100070000C94D8130C94D8130C94D8130C94D81354
:100080000C94D8130C94D8130C94D8130C94D81344
:100090000C94D8130C94D8130AE436E458E458E4CA
:1000A00058E458E458E458E458E458E458E458E470
:1000B00058E458E44EE446E43EE458E458E458E496
:1000C00058E458E458E458E430E416E41EE428E424
:1000D000084AD73B3BCE016E84BCBFFDC12F3D6CAF
:1000E00074319ABD56833DDA3D00C77F11BED9E415
:1000F000BB4C3E916BAAAABE000000803F05A84CF5
:10010000CDB2D44EB93836A9020C50B991868808C0
:100110003CA6AAAA2ABE000000803F004E414E49DC
:100120004E495459494E46CDCCCC3D0AD7233C17B5
:10013000B7D13877CC2B329595E6241FB14F0A0002
:100140000020410000C84200401C4620BCBE4CCAF2
:100150001B0E5AAEC59D74446F6E6520736176693F
:100160006E672066696C652E0A004D3239002020CA
:10017000506C616E6E657242756666657242797426
:1001800065733A20002046726565204D656D6F727B
:10019000793A2000436F6D70696C65643A204E6F48
:1001A0007620313220323031380A00207C204175EF
:1001B00074686F723A202844722E5068696C334418
:1001C000290A00323031382D30382D303100204CA2
:1001D00061737420557064617465643A2000312E37
:1001E000312E390A004D61726C696E0020536F66C2
:1001F00074776172652052657365740A00205761D7
:10020000746368646F672052657365740A002042E6
:10021000726F776E206F75742052657365740A0073
:100220002045787465726E616C2052657365740A3E
:1002300000506F77657255700A0073746172740AAA
:10024000005072696E7465722068616C7465642E0A
:10025000206B696C6C28292063616C6C6564210AD1
:10026000004B494C4C45442E20004B494C4C2063DC
:10027000617573656420627920746F6F206D75639A
:100280006820696E6163746976652074696D6520A4
:100290002D2063757272656E7420636F6D6D616E73
:1002A000643A200020746F6F206C6F6E6720657851
:1002B00074727573696F6E2070726576656E7465A1
:1002C000640A0020636F6C642065787472757369CA
:1002D0006F6E2070726576656E7465640A006F6B70
:1002E00000526573656E643A2000416476616E6306
:1002F00065204B3D003F4B2076616C7565206F7526
:1003000074206F662072616E67652028302D313051
:10031000292E0A003A200050726F6265205A204F41
:100320006666736574003F5A206F7574206F66208F
:1003300072616E676520282D3520746F2032302958
:100340000A00454550524F4D204F4B0A004265640C
:10035000204C6576656C696E6720004661696C6546
:100360006420746F20656E61626C65204265642054
:100370004C6576656C696E670A00426564204C6561
:1003800076656C20436F7272656374696F6E204D81
:1003900061747269783A004E6F2063617365206CF6
:1003A000696768740A0043290A0061626C65642009
:1003B000286D696E2074656D702000436F6C642039
:1003C0006578747275646573206172652000496E8A
:1003D00076616C69642065787472756465720A0070
:1003E00020643A0020693A0020703A0050726F622F
:1003F00065205A204F66667365743A200020466C6B
:100400006F773A2000205A00205900580020204DD4
:1004100061783A2000205A00205900580020204DD1
:10042000696E3A20004F6666004F6E2000536F667B
:100430007420656E6473746F70733A20004F666643
:1004400073657473206170706C69656400457272C5
:100450003A20546F6F206661722100546F6F2066DE
:1004600061722066726F6D207265666572656E637B
:100470006520706F696E740A00205400205200419C
:100480006363656C65726174696F6E3A2050004DEC
:1004900031343520533C696E6465783E206F757445
:1004A000206F662072616E67652028302D31290A21
:1004B000002F2F20003A004361703A005448455203
:1004C0004D414C5F50524F54454354494F4E0041AB
:1004D00055544F5245504F52545F53445F5354410B
:1004E00054555300454D455247454E43595F504181
:1004F0005253455200434153455F4C494748545F6E
:100500004252494748544E45535300544F47474C75
:10051000455F4C494748545300534F465457415246
:10052000455F504F574552004255494C445F504536
:100530005243454E54004C4556454C494E475F4446
:10054000415441005A5F50524F4245004155544F6B
:100550004C4556454C005052494E545F4A4F42005C
:1005600050524F4752455353004155544F524550F6
:100570004F52545F54454D5000564F4C554D4554C5
:1005800052494300454550524F4D00534552494151
:100590004C5F584F4E5F584F4646004649524D57A4
:1005A0004152455F4E414D453A4D61726C696E2036
:1005B000312E312E392028476974687562292053FD
:1005C0004F555243455F434F44455F55524C3A683F
:1005D000747470733A2F2F6769746875622E636F35
:1005E0006D2F4D61726C696E4669726D77617265CF
:1005F0002F4D61726C696E2050524F544F434F4CD7
:100600005F56455253494F4E3A312E30204D4143AB
:1006100048494E455F545950453A33442050726919
:100620006E7465722045585452554445525F434F8D
:10063000554E543A3120555549443A343063653665
:100640003164312D326564302D343533302D3833FB
:1006500030342D3535653365656161656266660ADE
:10066000003344205072696E746572204F66662EA6
:100670000020573A0042656420636F6F6C696E67B3
:100680002E2E2E004265642068656174696E672EA7
:100690002E2E0020573A004520436F6F6C696E671D
:1006A0002E2E2E00452048656174696E672E2E2E11
:1006B000006F6B004D3131332053004B494C4C459A
:1006C000442E20004543484F00494E464F004552B6
:1006D000524F52530044525952554E00434F4D4DC4
:1006E000554E49434154494F4E006F666600C4065B
:1006F000C906CE06D506DC0644454255473A0050A9
:10070000726F7465637465642050696E0A0000013D
:100710001C1D132FFFFFFFFF1E1F12FF14FFFFFF03
:1007200020211124FFFFFFFFFFFFFF0E10FFFFFF3F
:1007300022230DFFFFFF0E260F2C272569730025AE
:10074000696D20256973002569682025696D20255C
:10075000697300256964202569682025696D202555
:100760006973002569792025696420256968202539
:10077000696D20256973005072696E742074696D0B
:10078000653A200043757272656E742066696C6507
:100790003A2000456E642066696C65206C6973744C
:1007A0000A00426567696E2066696C65206C697332
:1007B000740A004E6F206D6F76652E00436C69637E
:1007C0006B20746F20726573756D652E2E2E002060
:1007D0005A3A200020593A200042656420583A20B5
:1007E000000A0A426564204C6576656C20436F728E
:1007F00072656374696F6E204D61747269783A0036
:10080000202844525952554E29004732392041750B
:10081000746F20426564204C6576656C696E670074
:100820003F2856296572626F7365206C6576656C2A
:1008300020697320696D706C61757369626C6520E5
:1008400028302D34292E0A00536C6565702E2E2E0B
:100850000047322F47332062616420706172616DFE
:1008600065746572730A00496E76616C696420650F
:10087000787472756465720A0041637469766520E4
:1008800045787472756465723A200020453A0020FC
:100890005A3A0020593A00583A002C20002C2000E7
:1008A000486F6D652058592066697273740A004854
:1008B0006F6D6520585920666972737400576172B4
:1008C0006E696E673A20486F6D696E672042756D7C
:1008D000702044697669736F72203C20310A0002EF
:1008E0000204627573793A207061757365642066DD
:1008F0006F7220696E7075740A00627573793A20A0
:1009000070617573656420666F7220757365720A15
:1009100000627573793A2070726F63657373696EE4
:10092000670A0050726F62696E67206661696C6564
:10093000640A0050726F62696E67206661696C6557
:100940006400205A3A200020593A20004265642071
:10095000583A2000486F6D65202573257325732054
:100960006669727374002066697273740A005A00B3
:1009700059005800486F6D65200020496E76616C03
:100980006964206578747275646572200053442030
:1009900072656164206572726F720A00446F6E65E1
:1009A000207072696E74696E672066696C650A00F2
:1009B0004B494C4C45442E200053544F5050454415
:1009C0002E20005072696E7465722073746F70709F
:1009D00065642064756520746F206572726F727330
:1009E0002E2046697820746865206572726F7220C7
:1009F000616E6420757365204D39393920746F201C
:100A0000726573746172742E202854656D706572FE
:100A100061747572652069732072657365742E2028
:100A20005365742069742061667465722072657301
:100A300074617274696E67290A004E6F204368659D
:100A4000636B73756D2077697468206C696E6520BF
:100A50006E756D6265722C204C617374204C696EEA
:100A6000653A20004E6F20436865636B73756D2097
:100A700077697468206C696E65206E756D62657249
:100A80002C204C617374204C696E653A20006368B9
:100A900065636B73756D206D69736D617463682C2C
:100AA000204C617374204C696E653A20004C696E6D
:100AB00065204E756D626572206973206E6F7420BB
:100AC0004C617374204C696E65204E756D62657261
:100AD0002B312C204C617374204C696E653A2000D8
:100AE0004D31313000656E7175657565696E6720D1
:100AF0002200FF01FF0000A0400000A04000000015
:100B00004000002043000011430000164300000095
:100B1000000000114300000000000020430000110D
:100B20004300001643000000000000000000000029
:100B300000000048420000484200008040000000E1
:100B4000007C3C3E5E2B3D3F2F5B5D3B2C2A225CB4
:100B5000004D33310043616E6E6F7420656E7465B5
:100B600072207375626469723A20006F70656E203E
:100B70006661696C65642C2046696C653A20006189
:100B800075746F25692E67006572726F72207772B7
:100B90006974696E6720746F2066696C650A004E1F
:100BA0006F74205344207072696E74696E670A0016
:100BB0005344207072696E74696E6720627974653F
:100BC000200044656C6574696F6E206661696C65B0
:100BD000642C2046696C653A200046696C65206487
:100BE000656C657465643A0057726974696E672054
:100BF000746F2066696C653A20006F70656E2066C0
:100C000061696C65642C2046696C653A20006F70E0
:100C1000656E206661696C65642C2046696C653A76
:100C2000200046696C652073656C65637465640AB1
:100C3000002053697A653A200046696C65206F7020
:100C4000656E65643A20002066696C653A2000662E
:100C50007265736800646F696E67004E6F7720007D
:100C6000454E4420535542524F5554494E450A0073
:100C70002220706F73002220706172656E743A22B8
:100C800000535542524F5554494E452043414C4C18
:100C9000207461726765743A22004B494C4C45449C
:100CA0002E2000747279696E6720746F2063616C06
:100CB0006C207375622D67636F64652066696C656F
:100CC00073207769746820746F6F206D616E79206E
:100CD0006C6576656C732E204D4158206C65766589
:100CE0006C2069733A004D3234004D323320257345
:100CF0000053442063617264206F6B0A006F70655B
:100D00006E526F6F74206661696C65640A00766F5D
:100D10006C756D652E696E6974206661696C6564B9
:100D20000A00534420696E6974206661696C0A0088
:100D3000286E6F2066696C65290043616E6E6F7462
:100D4000206F70656E2073756264697220003A0AC4
:100D50000020286D6D290020204D393030204B00B7
:100D60004C696E65617220416476616E63653A0A12
:100D70000020204D383531205A005A2D50726F62B4
:100D800065204F666673657400204400204900208A
:100D9000204D333031205000504944207365747425
:100DA000696E67733A0A002046002042002048001E
:100DB00020204D3134352053004D617465726961D6
:100DC0006C2068656174757020706172616D657406
:100DD0006572733A0A0020204D34323020530041AE
:100DE00075746F20426564204C6576656C696E672A
:100DF0003A0A00205A0020590020204D3230362077
:100E00005800486F6D65206F66667365743A0A0016
:100E1000204500205A00205900205800205400206E
:100E2000530020204D32303520510020453C6D616B
:100E3000785F655F6A65726B3E0020583C6D617833
:100E40005F785F6A65726B3E20593C6D61785F79AF
:100E50005F6A65726B3E205A3C6D61785F7A5F6AAB
:100E600065726B3E00416476616E6365643A205141
:100E70003C6D696E5F7365676D656E745F74696DF7
:100E8000655F75733E20533C6D696E5F6665656492
:100E9000726174653E20543C6D696E5F7472617658
:100EA000656C5F66656564726174653E0020540020
:100EB00020520020204D32303420500041636365C1
:100EC0006C65726174696F6E2028756E6974732F1A
:100ED0007332293A20503C7072696E745F616363AB
:100EE000656C3E20523C726574726163745F61632D
:100EF00063656C3E20543C74726176656C5F61631F
:100F000063656C3E0A00204500205A0020590020ED
:100F1000204D3230312058004D6178696D756D205B
:100F2000416363656C65726174696F6E2028756ECC
:100F30006974732F7332293A0A00204500205A0041
:100F400020590020204D3230332058004D617869FF
:100F50006D756D20666565647261746573202875B2
:100F60006E6974732F73293A0A00204500205A00D5
:100F700020590020204D3932205800537465707379
:100F80002070657220756E69743A0A0020204D3217
:100F900030302044300A0020204D323030204400D0
:100FA0002044697361626C65640A0046696C616D16
:100FB000656E742073657474696E67733A002020DF
:100FC0004D3134392043203B20556E6974732069BC
:100FD0006E2043656C736975730A002020473231B7
:100FE000202020203B0048617264636F64656420A8
:100FF00044656661756C742053657474696E6773BB
:10100000204C6F616465640A00DC050000DC0500AB
:1010100000DC050000102700000000FA420000FA82
:1010200042000070410000C8410000A0420000A042
:10103000420000C8430000C142290A0020627974BE
:1010400065733B2063726320002073746F72656464
:101050002073657474696E67732072657472696554
:10106000766564202800202863616C63756C617468
:10107000656429210A0020213D2000454550524F3A
:101080004D20435243206D69736D61746368202D58
:10109000202873746F7265642920002053697A6573
:1010A0003A2000496E6465783A2000204D61726CE8
:1010B000696E3D563535290A0028454550524F4D39
:1010C0003D00454550524F4D2076657273696F6EF5
:1010D000206D69736D617463682000290A002062C5
:1010E000797465733B20637263200053657474697F
:1010F0006E67732053746F726564202800454550F5
:10110000524F4D206461746173697A652065727213
:101110006F722E0A004572726F722077726974695D
:101120006E6720746F20454550524F4D210A006F65
:1011300070656E00545249474745524544003A2075
:10114000007A5F6D696E00795F6D617800785F6D20
:10115000696E005265706F7274696E6720656E64A7
:1011600073746F70207374617475730A00456E64D4
:1011700073746F70732025632025632025632025F9
:101180006300205A3A0020593A0020583A00656E10
:101190006473746F7073206869743A2000486F6DCF
:1011A000696E67206661696C656400556E6B6E6F71
:1011B000776E20636F6D6D616E643A20220020743B
:1011C0006F6F206C6F6E6720657874727573696FCE
:1011D0006E2070726576656E7465640A0020636FB8
:1011E0006C6420657874727573696F6E20707265B7
:1011F00076656E7465640A00FFFDFCFAF8F6F4F299
:10120000F0EEECEAE9E7E5E3E1E0DEDCDAD9D7D5B8
:10121000D4D2D0CFCDCBCAC8C7C5C3C2C0BFBDBC56
:10122000BAB9B7B6B4B3B2B0AFADACAAA9A8A6A5C7
:10123000A4A2A1A09E9D9C9A999897959493929010
:101240008F8E8D8B8A8988878684838281807F7E3A
:101250007D7B7A797877767574737271706F6E6D45
:101260006C6B6A696867666564636261605F5E5D36
:101270005C5B5A5958585756555453525150504F19
:101280004E4D4C4B4A4A49484746464544434242E4
:1012900041403F3E3E3D3C3B3B3A3938383736359E
:1012A00035343332323130302F2E2E2D2C2B2B2A49
:1012B00029292827272625252423232221212020E8
:1012C0001F1E1E1D1C1C1B1B1A1919181817161679
:1012D000151514131312121111100F0F0E0E0D0D00
:1012E0000C0C0B0A0A09090808070706060505047D
:1012F00004030302020100000000000100000001DD
:101300000000800055555500000040003333330085
:10131000AAAA2A004992240000002000C7711C00DC
:1013200099991900D1451700555515003BB1130087
:101330002449120011111100000010000F0F0F00BE
:10134000E3380E0043790D00CCCC0C00C3300C0008
:10135000E8A20B0064210B00AAAA0A00703D0A0053
:101360009DD80900427B090092240900DCD30800C3
:10137000888808001042080000000800F0C107003B
:101380008787070075500700711C07003EEB0600B9
:10139000A1BC06006990060066660600703E060065
:1013A0006118060017F4050074D105005BB0050054
:1013B000B2900500627205005555050078390500A8
:1013C000B81E0500050505004EEC040087D4040096
:1013D000A1BD040090A7040049920400C17D04004F
:1013E000EE690400C7560400444404005C32040063
:1013F0000821040041100400000004003FF0030035
:10140000F8E0030026D20300C3C30300CCB50300F9
:101410003AA803000A9B0300388E0300C081030032
:101420009F750300D0690300505E03001D53030045
:1014300034480300913D03003333030016290300B1
:10144000381F030097150300300C0300030303004B
:101450000BFA020049F10200BAE802005CE0020067
:101460002DD802002DD0020059C80200B0C00200E1
:1014700031B90200DAB10200AAAA0200A0A3020058
:10148000BC9C0200FA9502005C8F0200DF8802001B
:1014900082820200457C020027760200277002004B
:1014A000436A02007C640200D05E02003F590200E1
:1014B000C85302006563686F3A004572726F723AF2
:1014C00000205A3A0020593A0020436F756E74206C
:1014D000583A00232C0000B8220000561800003AA9
:1014E0000F0000B8080000B1040000710200003EC7
:1014F00001000024F4D43050C38E20C2A2401782D1
:101500008B7011127A910D816CD90AA861E108C71C
:10151000586607615143061E4B5D05C145A7041A75
:10152000411104093D9803713931034036DB0265EE
:10153000339102D4305402802E1D02632CEE0175CB
:101540002AC501B028A001102781018F2564012B35
:10155000244B01E0223401AC211F018D200D0180BC
:101560001FFC00841EED00971DDF00B81CD200E6B2
:101570001BC600201BBC00641AB200B219A8000AE6
:1015800019A0006A189900D117910040178B00B577
:1015900016840031167E00B31579003A157300C722
:1015A000146F0058146A00EE136600881363002558
:1015B000135E00C7125B006C12570015125400C175
:1015C00011510070114F0021114B00D61049008DB0
:1015D0001047004610440002104200C00F40008037
:1015E0000F3E00420F3C00060F3B00CB0E3800932D
:1015F0000E37005C0E3500270E3400F30D3200C1AB
:101600000D3100900D3000600D2E00320D2D0005C3
:101610000D2C00D90C2B00AE0C2900850C29005C88
:101620000C2700350C27000E0C2600E80B2400C404
:101630000B2400A00B23007D0B23005A0B21003943
:101640000B2100180B2000F80A1F00D90A1E00BB4E
:101650000A1E009D0A1D00800A1D00630A1C004727
:101660000A1B002C0A1B00110A1A00F7091A00DDD8
:10167000091900C4091900AB091900920917007B68
:10168000091800630917004C0916003609160020D6
:101690000916000A091500F5081500E0081400CC29
:1016A000081400B8081400A4081400900813007D62
:1016B0000812006B08130058081200460812003484
:1016C000081100230811001208110001081100F090
:1016D000071000E0071000D0071000C0071000B08E
:1016E000070F00A107100091070E0083070F007479
:1016F000070F0065070E0057070E0049070E003B55
:10170000070D002E070E0020070D0013070D000621
:10171000070D00F9060C00ED060D00E0060C00D4E4
:10172000060C00C8060C00BC060C00B0060C00A499
:10173000060B0099060C008D060B0082060B007745
:10174000060B006C060B0061060A0057060B004CE6
:10175000060A0042060A0038060A002E060A00247D
:10176000060A001A060A001006090007060A00FD0C
:10177000050900F4050900EB050900E2050900D997
:10178000050900D0050900C7050900BE050900B517
:10179000050800AD050800A50509009C0508009492
:1017A0000508008C050800840508007C0508007405
:1017B0000508006C050700650508005D0507005673
:1017C0000508004E050700470507004005080038DA
:1017D000050700310507002A050700230507001C3F
:1017E000050600160507000F05070008050600029C
:1017F000050700FB040600F5040700EE040600E8F8
:10180000040600E2040700DB040600D5040600CF4E
:10181000040600C9040600C3040600BD040600B7A0
:10182000040600B1040500AC040600A6040600A0EE
:101830000405009B04060095040500900406008A38
:1018400004050085040500800406007A040500757F
:10185000040500700405006B0405006604050061C2
:101860000405005C04050057040500520405004D02
:1018700004050048040500430405003E0404003A42
:1018800004050035040500300404002C040500277D
:10189000040400230405001E0404001A04040016B6
:1018A000040500110404000D0404000904050004EB
:1018B00004040000040400FC030400F8030400F422
:1018C000030400F0030400EC030400E8030400E454
:1018D000030400E0030400DC030400D8030400D484
:1018E000030400D0030400CC030400C8030300C5B4
:1018F00003030024F404D9201BC40C5C0E9804C418
:10190000095F0265077101F405F900FB04B30048A3
:10191000048700C10369005803550003034500BE56
:10192000023A008402310053022A002902250004F1
:10193000022000E4011C00C8011900AF0117009843
:1019400001140084011300710110006101100051A5
:10195000010E0043010D0036010B002B010B00208E
:10196000010B00150109000C01090003010800FB2F
:10197000000800F3000800EB000700E4000600DEAA
:10198000000600D8000600D2000600CC000500C703
:10199000000500C2000500BD000400B9000400B548
:1019A000000400B1000400AD000400A9000400A57B
:1019B000000300A20003009F0004009B00030098A6
:1019C0000003009500020093000300900003008DC7
:1019D0000002008B000300880002008600020084E1
:1019E000000300810002007F0002007D0002007BF6
:1019F0000002007900020077000100760002007406
:101A000000020072000100710002006F0002006D10
:101A10000001006C0002006A00010069000200671A
:101A20000001006600010065000100640002006220
:101A300000010061000100600001005F0002005D24
:101A40000001005C0001005B0001005A0001005928
:101A50000001005800010057000100560001005528
:101A60000001005400010053000000530001005227
:101A700000010051000100500001004F0001004E24
:101A80000000004E0001004D0001004C0001004B21
:101A90000000004B0001004A00010049000100481D
:101AA0000000004800010047000100460000004619
:101AB0000001004500000045000100440001004312
:101AC000000000430001004200000042000100410C
:101AD00000000041000100400001003F0000003F05
:101AE0000001003E0000003E0001003D0000003DFE
:101AF0000001003C0000003C0000003C0001003BF5
:101B00000000003B0001003A0000003A00010039EB
:101B100000000039000100380000003800000038E3
:101B200000010037000000370001003600000036D9
:101B300000000036000100350000003500000035CF
:101B400000010034000000340000003400010033C4
:101B500000000033000000330001003200000032BA
:101B600000000032000100310000003100000031AF
:101B70000001003000000030000000300001002FA4
:101B80000000002F0000002F0000002F0001002E99
:101B90000000002E0000002E0001002D0000002D8E
:101BA0000000002D0000002D0001002C0000002C82
:101BB0000000002C0000002C0001002B0000002B76
:101BC0000000002B0000002B0001002A0000002A6A
:101BD0000000002A0000002A00010029000000295E
:101BE0000000002900000029000000290001002851
:101BF0000000002800000028000000280000002845
:101C00000001002700000027000000270000002737
:101C1000000000270001002600000026000000262A
:101C2000000000260000002600010025000000251D
:101C30000000002500000025000000250000002510
:101C40000001002400000024000000240000002403
:101C500000000024000100230000002300000023F6
:101C600000000023000000230000002300000023E8
:101C700000010022000000220000002200000022DB
:101C800000000022000000220001002100000021CD
:101C900000000021000000210000002100000021C0
:101CA00000000021000100200000002000000020B2
:101CB00000000020000000200000002000000020A4
:101CC000000000200001001F0000001F0000001F96
:101CD0000000001F0000001F0000001F0000001F88
:101CE0000001001E0000001E0000001E0000001E7B
:101CF0000000002042403A0020403A00202F004DD2
:101D0000383420582059205A204500546865726D97
:101D1000616C2052756E61776179004531205448BD
:101D200045524D414C2052554E4157415900424574
:101D30004420544845524D414C2052554E41574144
:101D400059004B494C4C45442E2000202D20496E13
:101D500076616C6964206578747275646572206E52
:101D6000756D62657220210A0048656174696E674D
:101D7000206661696C656400426564206865617411
:101D8000696E67206661696C6564004865617469A5
:101D90006E67206661696C65640045312048656145
:101DA00074696E67206661696C6564004D494E54C4
:101DB000454D5020747269676765726564004531EE
:101DC000204572723A204D494E54454D500045729F
:101DD000723A204D494E54454D5020424544004DE5
:101DE000415854454D502074726967676572656447
:101DF000004531204572723A204D415854454D50AE
:101E0000004572723A204D415854454D502042458C
:101E100044006265640A002C2073797374656D2038
:101E200073746F7070656421204865617465725FBA
:101E300049443A20002CFFFFFFFFFF000101010190
:101E40000123646566696E652044454641554C54DE
:101E50005F4B64200023646566696E6520444546D7
:101E600041554C545F4B69200023646566696E657B
:101E70002044454641554C545F4B70200050494426
:101E8000204175746F74756E652066696E6973683C
:101E90006564212050757420746865206C617374CA
:101EA000204B702C204B6920616E64204B642063B2
:101EB0006F6E7374616E74732066726F6D206265ED
:101EC0006C6F7720696E746F20436F6E66696775FB
:101ED000726174696F6E2E680A0050494420417522
:101EE000746F74756E65206661696C656421207419
:101EF000696D656F75740A00546865726D616C2058
:101F000052756E6177617900453120544845524DD4
:101F1000414C2052554E4157415900486561746902
:101F20006E67206661696C656400453120486561B3
:101F300074696E67206661696C656400504944206D
:101F40004175746F74756E65206661696C65642196
:101F50002054656D706572617475726520746F6F61
:101F600020686967680A00204B643A2000204B69AA
:101F70003A2000204B703A20000A20436C617373B2
:101F8000696320504944200A002054753A200020FB
:101F90004B753A2000206D61783A2000206D696E03
:101FA0003A200020643A200020626961733A2000E0
:101FB000504944204175746F74756E652073746167
:101FC00072740A00504944204175746F74756E65CF
:101FD000206661696C6564212042616420657874C3
:101FE0007275646572206E756D6265720A0010000C
:101FF000C90210012C014001220170011801B00139
:102000000E01F00104015002FA00B002F0003003AA
:10201000E600D003DC009004D2007005C800A006E2
:10202000BE000008B400B009AA00D00BA000600EEA
:10203000960060118C000015820020197800C01DE8
:102040006E00A0226400B0275A00902C500000318E
:102050004600E0343C0010383200903A2800603CE2
:102060001E00A03D1400803E0A00203F00007001C9
:102070002C0190012701B0012201C0011D01F001D6
:1020800018011002130130020E01600209019002D2
:102090000401C002FF000003FA004003F5008003C2
:1020A000F000D003EB002004E6007004E100E0043F
:1020B000DC004005D700C005D2004006CD00D006A8
:1020C000C8008007C3003008BE00F008B900C0098E
:1020D000B400B00AAF00B00BAA00D00CA500000EEF
:1020E000A000500F9B00C0109600501291000014E9
:1020F0008C00C0158700B0178200B0197D00D01B7E
:102100007800001E730040206E0090226900F024C9
:10211000640040275F0090295A00E02B5500102EE4
:10212000500020304B0010324600E0334100903523
:102130003C001037370070383200A0392D00B03A1B
:102140002800A03B2300603C1E00103D1900903D7C
:102150001400103E0F00703E0A00C03E0500003F14
:102160000000403FFBFF803FF6FFC03FF1FF052E20
:102170002E000452656672657368004D61696E00D9
:1021800046696C2E204469612E0046696C2E2044FD
:1021900069612E004520696E206D6D33004F6666C3
:1021A000004F6E2000416476616E6365204B0041F4
:1021B0006476616E6365204B00436F6E74726F6C62
:1021C0000050726F6265205A204F66667365740016
:1021D000436F6E74726F6C005049442D4400504937
:1021E000442D44005049442D49005049442D490094
:1021F0005049442D50005049442D500020022046A3
:102200006163740020022046616374002002204D47
:102210006178002002204D6178002002204D696E17
:10222000002002204D696E004175746F74656D70F9
:10223000004F6666004F6E200046616E2073706529
:1022400065640046616E2073706565640042656474
:1022500000426564004E6F7A7A6C65004E6F7A7A40
:102260006C6500436F6E74726F6C00526573746FAF
:102270007265206661696C73616665004C6F6164AC
:102280002073657474696E67730053746F72652090
:1022900073657474696E67730046696C616D656E11
:1022A00074004D6F74696F6E0054656D7065726176
:1022B00074757265004D61696E004578747275645D
:1022C0006572004D6F7665205A004D6F7665205916
:1022D000004D6F7665205800507265706172650020
:1022E0004D6F766520302E316D6D004D6F76652017
:1022F000316D6D004D6F76652031306D6D004D6F25
:1023000076652061786973004578747275646572CA
:10231000004D6F7665205A004D6F76652059004D4F
:102320006F76652058004578747275646572004D4B
:102330006F7665205A004D6F76652059004D6F7697
:1023400065205800507265686561742041425300F1
:102350005072656865617420504C4100436F6F6C2A
:10236000646F776E0044697361626C652073746595
:102370007070657273004D383400426564204C659E
:1023800076656C696E67004175746F20686F6D6566
:1023900000473238004D6F76652061786973004DD3
:1023A00061696E0053746F72652073657474696E31
:1023B0006773004C6F61642073657474696E677332
:1023C0000050726F6265205A204F66667365740014
:1023D000426564204C6576656C696E67004F666681
:1023E000004F6E20004C6576656C20626564004786
:1023F00032380A47323900473239004175746F204C
:10240000686F6D65004732380050726570617265A3
:1024100000507265686561742041425320426564D2
:1024200000507265686561742041425320456E64B6
:1024300000507265686561742041425300507265B6
:1024400070617265005072656865617420504C411E
:1024500020426564005072656865617420504C418B
:1024600020456E64005072656865617420504C416F
:1024700000507265706172650050726F6265205A1B
:10248000204F666673657400466C6F7700466C6F0C
:10249000770046616E2073706565640046616E204A
:1024A00073706565640042656400426564004E6F48
:1024B0007A7A6C65004E6F7A7A6C65005370656548
:1024C00064005370656564004D61696E00496E6912
:1024D000742E2053442063617264004D3231004EEB
:1024E0006F2053442063617264004368616E6765C6
:1024F0002053442063617264004D32310050726990
:102500006E742066726F6D2053440053746F702098
:102510007072696E7400526573756D6520707269B2
:102520006E74005061757365207072696E7400433B
:102530006F6E74726F6C00507265706172650054DA
:10254000756E6500496E666F2073637265656E0017
:102550005072696E742061626F72746564003344F6
:10256000205072696E7465722052656164792E0024
:102570005072696E74696E672E2E2E005072696EED
:1025800074207061757365640025753A2530327565
:1025900000253032753A2530327500202020200089
:1025A000202020202020002D2D2D00534400001C31
:1025B0001F11111F00000006191803130C00040E50
:1025C0001F041C000000000E1315110E00001C104B
:1025D000181705060500040A0A0A0A11110E0C1242
:1025E000120C00000000001F1511151F0000507292
:1025F0006F6265205A204F666673657400506C6583
:10260000617365207265736574005052494E54457C
:10261000522048414C54454400012902290429080C
:10262000291029202940298029012C022C01260269
:1026300026042608261026202640268026402C80A8
:102640002C0123022304230823102320234023806A
:102650002301200220042008201020202040208078
:1026600020102C202C012F022F042F082F102F2098
:102670002F402F802F7EFE7EFD7EFB7EF77EEF7E3D
:10268000DF7EBF7E7F0001000036271200020000BF
:10269000F3264300030000EF260401030904D526B6
:1026A0001802030904BD261603030904AF260C0C07
:1026B00003310032003300340035000000160355AA
:1026C0000053004200200053006500720069006161
:1026D000006C00000018035400650065006E007374
:1026E0000079006400750069006E006F000000044E
:1026F00003090409024300020100C032090400007A
:10270000010202010005240010010524010001045A
:10271000240206052406000107058203080040097B
:10272000040100020A000000070503024000000740
:102730000584024000001201000202000020C016C1
:1027400083047202010203010001C102018036010B
:1027500081361F373C93BBBBDFEA233711241FBEF2
:10276000CFEFD0E2DEBFCDBF12E0A0E0B1E0E8E500
:10277000FEEE01E00BBF02C007900D92A034B1073E
:10278000D9F722E1A0E4B2E001C01D92A43CB20757
:10279000E1F713E1CDEAD3E104C02197FE010E94E5
:1027A00067EBC93AD107C9F70E949CE30C941FF765
:1027B0000C9400004F925F926F927F928F929F9243
:1027C000AF92BF92CF92DF92EF92FF92CF934B01E5
:1027D0005C0169017A0120E030E040EA51E40E94A6
:1027E0008FEB2B013C012FE632E143E85AEB0E94CC
:1027F0006CEE87FD48C022E430E040E253E4C301C0
:10280000B2010E9469EC18160CF43DC02FE632E1CB
:1028100043E85AEBC701B6010E946CEE87FD33C056
:1028200022E430E041E153E4C701B6010E9469ECC3
:1028300018164CF124EF3DEF4FE951E4C501B40106
:102840000E946CEE87FD1FC022E430E046E153E4B5
:10285000C501B4010E9469EC1816ACF027EE3BEFFD
:102860004FE151E4C701B6010E946CEE87FD0BC039
:10287000C1E022E430E046E053E4C701B6010E9423
:1028800069EC18160CF4C0E08C2FCF91FF90EF90FC
:10289000DF90CF90BF90AF909F908F907F906F9080
:1028A0005F904F900895FB0101900020E9F7319768
:1028B000AF01461B570BDC01ED91FC910280F381C7
:1028C000E02D0994CF93DF931F92CDB7DEB76983D4
:1028D000DC01ED91FC910280F381E02D41E050E0BC
:1028E000BE016F5F7F4F09950F90DF91CF910895E3
:1028F000FF920F931F93CF93DF93F82E092F162F7C
:10290000E7EBF4E06491EF012196662329F088EB70
:1029100092E1D8DFFE01F6CFEF2DF02F6491EF01A9
:102920002196662329F088EB92E1CCDFFE01F6CFF9
:10293000E5EBF4E06491EF012196662329F088EB42
:1029400092E1C0DFFE01F6CF412F50E060E070E081
:1029500088EB92E10E94E8E26AE088EB92E1DF9185
:10296000CF911F910F91FF90ADCF0FB6F89480914A
:10297000AD129091AE12A091AF12B091B0120FBEF5
:102980008093C1029093C202A093C302B093C40289
:1029900008954F925F926F927F92AF92BF92CF92C3
:1029A000DF92EF92FF92CF93DF93EB01FC01608106
:1029B0007181828193812CE3C22ED12CE12CF12CE8
:1029C000A70196010E9429EBB62EA72ECA01B901D4
:1029D000A70196010E9429EB6B017C01CA01B90194
:1029E00028E130E040E050E00E9429EB2B013C015F
:1029F000C9016DE671E00E9402EB61157105D9F025
:102A0000AF92BF92DF92CF925F924F929F938F933C
:102A10007F936F9383E697E09F938F93DF93CF939A
:102A20000E9405F48DB79EB70E960FB6F8949EBF20
:102A30000FBE8DBF61C00097C9F0AF92BF92DF9209
:102A4000CF925F924F929F938F9383E597E09F93EE
:102A50008F93DF93CF930E9405F4EDB7FEB73C96BA
:102A60000FB6F894FEBF0FBEEDBF46C0411451042F
:102A700061047104B9F0AF92BF92DF92CF925F927E
:102A80004F9287E497E09F938F93DF93CF930E94B9
:102A900005F48DB79EB70A960FB6F8949EBF0FBE89
:102AA0008DBF2AC0C114D104E104F104A9F0AF9292
:102AB000BF92DF92CF928FE397E09F938F93DF9344
:102AC000CF930E9405F4EDB7FEB738960FB6F89491
:102AD000FEBF0FBEEDBF10C0AF92BF928BE397E079
:102AE0009F938F93DF93CF930E9405F40F900F90E5
:102AF0000F900F900F900F90DF91CF91FF90EF907C
:102B0000DF90CF90BF90AF907F906F905F904F908D
:102B1000089581548A3108F040C0A82FB0E0409158
:102B2000600950916109609162097091630904C064
:102B300076956795579547958A95D2F740FF2DC0B2
:102B4000E0916B09F0916C09AA5BB64F8C918823D8
:102B5000E1F0E80FF11D808190ED980F9A3080F040
:102B60008E3229F4818180538A3078F409C08D3205
:102B700011F08B3251F4818190ED980F9A3018F456
:102B80009E2F8F2F04C08E3251F090E080E0909302
:102B900067098093680981E0089580E00895828143
:102BA00080538A3090F7ECCFB4DF882341F081E086
:102BB0002091670930916809232B09F480E008957A
:102BC0000F931F93CF9380916709909168090097A5
:102BD00011F1FC018F01C1912C2F2F7DA9F0C5347B
:102BE00011F0C536B9F7F801108260E070E080910D
:102BF0006709909168090E9471EFF801C083562F10
:102C0000472F382F292F0BC060E070E0CF911F9124
:102C10000F910C9471EF50E040E030E020E0652F20
:102C2000742F832F922FCF911F910F910895809130
:102C3000670990916809009731F04AE050E060E040
:102C400070E00C94D7F060E070E0CB0108958091C3
:102C5000670990916809009731F04AE050E060E020
:102C600070E00C94FFF160E070E0CB010895DFDFCD
:102C700097FD0AC0DCDF6F3F71058105910509F002
:102C80002CF4D5DF862F089580E008958FEF089506
:102C90008091670990916809892B31F0E8DF91E014
:102CA000811103C090E001C091E0892F08950F9336
:102CB0001F93CF93DF93CDB7DEB72C970FB6F89461
:102CC000DEBF0FBECDBFE6EAF4E080859185A28528
:102CD000B38544815581668177810081118122818C
:102CE000338109871A872B873C874D835E836F83E7
:102CF000788789839A83AB83BC83AE014F5F5F4F34
:102D0000BE016B5F7F4FCE0109960E944B8222EB82
:102D100034E0AE014F5F5F4FBE016B5F7F4FCE016E
:102D200009960E94EC902C960FB6F894DEBF0FBE69
:102D3000CDBFDF91CF911F910F9108952F923F92B8
:102D40004F925F926F927F929F92AF92BF92CF927B
:102D5000DF92EF92FF920F931F93CF93DF93CDB744
:102D6000DEB764970FB6F894DEBF0FBECDBF2A0161
:102D70003B01902EA12E6901082F10E0F801EE50C2
:102D8000F54FE491BB24B3941E160CF4B12CFF2430
:102D9000F39420E030E0A901C301B2010E946CEE7F
:102DA00018160CF0F12C000F111F000F111FC80195
:102DB0008A559B4F1C01FC011082118212821382E2
:102DC00076DFF1014082518262827382E090CA0212
:102DD00020E030E0A901692D7A2DC6010E9469EC3E
:102DE000811108C0F801EF5CF44F85919591A59190
:102DF000B49103C0892D9A2DD601898B9A8BAB8B08
:102E0000BC8B8091AE049091AF04A091B004B091BE
:102E1000B1044091AA045091AB046091AC0470914C
:102E2000AD040091A6041091A7042091A80430914C
:102E3000A9040D871E872F87388B49875A876B8790
:102E40007C878D839E83AF83B88719821A821B8209
:102E50001C82AE014B5F5F4FBE01675F7F4FCE01AB
:102E60000D960E944B82CE0101966C018E010F5E81
:102E70001F4F22EB34E0AE014B5F5F4FBE01675F37
:102E80007F4F0C960E940A900E94E783BF100E9419
:102E9000E97664960FB6F894DEBF0FBECDBFDF9122
:102EA000CF911F910F91FF90EF90DF90CF90BF9047
:102EB000AF909F907F906F905F904F903F902F903A
:102EC000089562EB74E083E00C94129210928B04EC
:102ED0001092890410928A04089590918904E92F30
:102EE000F0E0E855FD4F80839F5F943018F4909395
:102EF000890402C01092890480918B048F5F8093B3
:102F00008B040895CF93FC0180818B33A1F08091D5
:102F10008B04843080F4C62FBF018091890420E6A1
:102F2000829FC0011124875F9C4F0E94D6F38C2F93
:102F3000D4DF81E001C080E0CF910895EF92FF924D
:102F40001F93CF93DF937C0160E0DCDF182F882391
:102F5000C9F0E4EBF4E16491EF012196662329F0D6
:102F600088EB92E1AFDCFE01F6CFB70185EE9AE087
:102F70000E94409362E288EB92E1A4DC6AE088EB75
:102F800092E1A0DC812FDF91CF911F91FF90EF9014
:102F90000895DF92EF92FF920F931F93CF93DF93E9
:102FA000CDB7DEB76E970FB6F894DEBF0FBECDBFBC
:102FB00060910703709108036115710541F14DE1BE
:102FC00050E0CE0101967C010E9465F31E8EF70150
:102FD0008F010E191F09D190DD2019F09AE0D91246
:102FE000F7CFF701E00FF11F1082C701A7DF882399
:102FF00071F0DD20A9F00F5F1F4F809107039091C2
:103000000803080F191F109308030093070381E0BA
:103010002091070330910803232B29F480E003C09B
:1030200000E010E0F0CF6E960FB6F894DEBF0FBE52
:10303000CDBFDF91CF911F910F91FF90EF90DF9067
:1030400008959093080380930703A3CFEF92FF9214
:103050000F931F93CF93DF937C0184E5A5DDD82FD9
:10306000882369F104DEC82F18162CF5E4EBF4E18F
:1030700064918F010F5F1F4F662329F088EB92E167
:1030800021DCF801F5CF6DE488EB92E11BDCA701B0
:1030900060E070E020E088EB92E10E948CE26C2F0F
:1030A000CC0F770B8AE799E00E9468936AE088EB7F
:1030B00092E108DC08C08093BC02D0E004C080919B
:1030C000CA028093BC028D2FDF91CF911F910F9187
:1030D000FF90EF9008950F931F93CF93DF9394E0A9
:1030E000899FE00111248E0107521D4FFE01EB5113
:1030F000FD4FDE01AF50BD4F2D913D914D915C9143
:1031000060817181828193810E9490EBF8016083DC
:10311000718382839383FE01EB5DF44F85919591DA
:10312000A591B491FE01E353FD4F80839183A28367
:10313000B383FE01E75EF44F85919591A591B4911B
:10314000C55FDE4F88839983AA83BB83DF91CF91CC
:103150001F910F910895CF92DF92EF920F931F93DB
:10316000CF93DF93CDB7DEB760970FB6F894DEBF8D
:103170000FBECDBFE090CA02E6EAF4E080859185FB
:10318000A285B38544815581668177810081118153
:10319000228133810D871E872F87388B49875A8775
:1031A0006B877C878D839E83AF83B88719821A8251
:1031B0001B821C82AE014B5F5F4FBE01675F7F4F7A
:1031C000CE010D960E944B82CE0101966C0109E161
:1031D00011E022EB34E0AE014B5F5F4FBE01675F51
:1031E0007F4F0C960E940A9060960FB6F894DEBF4F
:1031F0000FBECDBFDF91CF911F910F91EF90DF9068
:10320000CF9008954F925F926F927F928F929F928C
:10321000AF92BF92CF92DF92EF92FF920F931F93E4
:10322000CF93DF93CDB7DEB72C970FB6F894DEBF00
:103230000FBECDBF6D837E838F83988729873A87A2
:103240004B875C87470158013601809119019091A5
:103250001A01A0911B01B0911C0189839A83AB8351
:10326000BC83D601CD90DD90ED90FC9020E030E065
:10327000A901C701B6010E9469EC811106C0E9E30A
:10328000FBE0C590D590E590F490A5019401609184
:10329000AE047091AF048091B0049091B1040E948B
:1032A00069EC87FF11C0C0921901D0921A01E09217
:1032B0001B01F0921C018092AE049092AF04A09288
:1032C000B004B092B10447DFF301408051806280C6
:1032D000738020E030E0A901C301B2010E9469ECD3
:1032E000811108C0409001015090020160900301DB
:1032F000709004014092190150921A0160921B01D2
:1033000070921C018D819E81AF81B8858093A60447
:103310009093A704A093A804B093A90489859A85E3
:10332000AB85BC858093AA049093AB04A093AC04B6
:10333000B093AD0410DFA50194016091AE047091CB
:10334000AF048091B0049091B1040E946CEE181605
:103350008CF4C0921901D0921A01E0921B01F092F4
:103360001C018092AE049092AF04A092B004B0927F
:10337000B104F1DE0E94E78389819A81AB81BC812F
:103380008093190190931A01A0931B01B0931C0123
:103390002C960FB6F894DEBF0FBECDBFDF91CF9154
:1033A0001F910F91FF90EF90DF90CF90BF90AF9063
:1033B0009F908F907F906F905F904F900895CF92E5
:1033C000DF92EF92FF920F931F936B01FC01E0805D
:1033D000F18002811381E6EAF4E02481358146819F
:1033E000578160817181828193810CDF1F910F91E0
:1033F000FF90EF90DF90CF900895CF92DF92EF9201
:10340000FF920F931F936A01E090AE04F090AF0417
:103410000091B0041091B104FB01208131814281FF
:103420005381FC016081718182819381EBDE1F9168
:103430000F91FF90EF90DF90CF9008958091190148
:1034400090911A01A0911B01B0911C01809303037C
:1034500090930403A0930503B09306038091170192
:1034600090911801909302038093010384E690E009
:103470009093180180931701089580910303909110
:103480000403A0910503B091060380931901909362
:103490001A01A0931B01B0931C018091010390912C
:1034A000020390931801809317010895EF92FF9201
:1034B0001F93CF93DF93882329F0D0919504D09563
:1034C000D17001C0D0E0662341F01091950411FB4A
:1034D000882780F911E0182701C010E0442341F04B
:1034E000C0919504C2FB882780F9C1E0C82701C0BC
:1034F000C0E0D11105C0111103C0CC2309F486C06E
:10350000E4EBF4E164917F018FEFE81AF80A662397
:1035100029F088EB92E1D6D9F701F4CFE4E7F9E09E
:1035200064917F019FEFE91AF90A662329F088EB7D
:1035300092E1C8D9F701F4CFDD2371F0E2E7F9E0B9
:1035400064917F018FEFE81AF80A662329F088EB6F
:1035500092E1B8D9F701F4CF112371F0E0E7F9E077
:1035600064917F019FEFE91AF90A662329F088EB3D
:1035700092E1A8D9F701F4CFC11103C0E6E6F9E062
:103580000EC0EEE6F9E064917F018FEFE81AF80AC9
:103590006623A1F388EB92E195D9F701F4CF64910A
:1035A0007F019FEFE91AF90A662329F088EB92E17F
:1035B00089D9F701F4CFC11103C044EE51E002C034
:1035C00044ED51E0111103C024EE31E002C026EDBC
:1035D00031E0D11103C084EE91E002C088ED91E0AA
:1035E0005F934F933F932F939F938F9384E599E03D
:1035F0009F938F931F920E944BB98DB79EB70996E8
:103600000FB6F8949EBF0FBE8DBFC1E08C2FDF9127
:10361000CF911F91FF90EF900895BF92CF92DF92CC
:10362000EF92FF920F931F93CF93DF93CDB7DEB747
:1036300028970FB6F894DEBF0FBECDBF909140091A
:10364000981709F47AC0B82E882309F453C080E093
:1036500090E0A0EAB0E48D839E83AF83B887C090EA
:10366000B802D090B902E090BA02F090BB0220E01C
:1036700030E0A901C701B6010E9469EC87FF0CC0C8
:10368000A701960160E070E080EA90E40E948FEB71
:103690006D837E838F83988720E030E046E153E49A
:1036A0006D817E818F8198850E946CEE181644F49E
:1036B00080E090E0A6E1B3E48D839E83AF83B8877A
:1036C0002091AE043091AF044091B0045091B10408
:1036D0006D817E818F8198850E946CEE181654F45E
:1036E00019821A821B821C82BE016F5F7F4FCE013E
:1036F000059665DE6091A6047091A7048091A804E8
:103700009091A9042091AA043091AB044091AC049B
:103710005091AD0419821A821B821C82E090AE0483
:10372000F090AF040091B0041091B104FE01319605
:103730006F0168DD8B2D0E94F47680E028960FB62D
:10374000F894DEBF0FBECDBFDF91CF911F910F91D7
:10375000FF90EF90DF90CF90BF9008954F925F92CF
:103760006F927F928F929F92AF92BF92CF92DF9291
:10377000EF92FF920F931F93CF93C82FE82EF12C57
:10378000F701EE50F54FB490823021F481E045DF2F
:10379000811107C16701CC0CDD1CCC0CDD1CF601CE
:1037A000EF5FF44F45905590659074906B2DBB0C76
:1037B000770B880B990B0E940BED4B015C0120E00D
:1037C00030E040EC5FE3C301B2010E94A7EEA50127
:1037D00094010E94A7EEAB01BC0100E010E098014B
:1037E0008C2FACDAC23041F0F601EB50F54F259149
:1037F00035914591549104C020E030E040E450E41C
:10380000C501B4010E94A7EE4B015C0120E030E04D
:10381000A9010E9469EC882309F45CC0C23021F040
:1038200000E010E0980104C000E010E020E830E47F
:10383000B501A40170588C2F81DAC23009F439C067
:10384000F701E152F74F849181111DC0E4EBF4E1DF
:1038500064917F018FEFE81AF80A662329F088EB5C
:1038600092E130D8F701F4CFEDEBF8E064917F01FD
:103870008FEFE81AF80A662329F088EB92E122D844
:10388000F701F4CF8AE0F601EF5CF44F45905590D4
:1038900065907490682F70E080E090E00E940BEDDE
:1038A0009B01AC01C301B2010E9470EC2B013C01F1
:1038B00005C0412C512C612C90E4792EA501940176
:1038C000C501B4010E9490EBAB01BC0193018201E0
:1038D0008C2F34DA81E090E00C2E01C0880F0A941E
:1038E000EAF790919404982B909394049091950406
:1038F000892B80939504F601EF50FD4F10821182C1
:10390000128213828C2FE7DBF601E35FF44F85917F
:103910009591A591B491F601EA55FB4F808391836F
:10392000A283B383C230D1F42091B8023091B9029E
:103930004091BA025091BB026091AE047091AF0405
:103940008091B0049091B1040E948FEB6093AE041B
:103950007093AF048093B0049093B104A8D9F6019A
:10396000EA56FB4FD601AA55BB4F8D919D910D9004
:10397000BC91A02D80839183A283B383C23089F44C
:1039800080E0CF911F910F91FF90EF90DF90CF904B
:10399000BF90AF909F908F907F906F905F904F906F
:1039A0003CCECF911F910F91FF90EF90DF90CF9081
:1039B000BF90AF909F908F907F906F905F904F904F
:1039C000089581E00895AF92BF92CF92DF92EF9277
:1039D000FF920F931F93CF93DF938CEFA82E81E07C
:1039E000B82E96E9E92E94E0F92E06EA14E029EDC6
:1039F000C22E22E0D22EC0E0D0E0F50181915F011D
:103A000088D8882319F1DCD8FE01E350FD4F2081CE
:103A1000211104C02091C902222341F0F801208124
:103A20003181428153810E9490EB0AC0C330D1059D
:103A300039F0F60120813181428153810E948FEB60
:103A4000F70160837183828393830AC0F8018081C8
:103A50009181A281B381F70180839183A283B38393
:103A60002196F4E0EF0EF11C0C5F1F4F84E0C80EAE
:103A7000D11CC430D10509F0C0CF86E495D8882385
:103A8000B9F09ED820E030E0A9010E946CEE181633
:103A90007CF496D820E030E040E752E40E9470ECDD
:103AA0006093190170931A0180931B0190931C017C
:103AB000DF91CF911F910F91FF90EF90DF90CF900A
:103AC000BF90AF900895CF92DF92EF92FF920F9345
:103AD0001F93CF93DF930FB6F894C090AD12D090A0
:103AE000AE12E090AF12F090B0120FBE8091C702FC
:103AF000811174C080910001882309F46FC0809106
:103B0000A702882309F46AC04091A3025091A4023D
:103B10006091A5027091A60297018601041B150B06
:103B2000260B370B37FD6DC0833031F134F4813013
:103B30000CF454C0E4EBF4E106C0843009F04EC04C
:103B4000E4EBF4E133C06491EF012196662331F098
:103B500088EB92E10E946214FE01F5CFE1E1F9E009
:103B60006491EF012196662309F438C088EB92E155
:103B70000E946214FE01F4CFE4EBF4E16491EF01E2
:103B80002196662331F088EB92E10E946214FE01D7
:103B9000F5CFEAEFF8E06491EF0121966623F1F0AA
:103BA00088EB92E10E946214FE01F5CF6491EF016F
:103BB0002196662331F088EB92E10E946214FE01A7
:103BC000F5CFE2EEF8E06491EF012196662331F043
:103BD00088EB92E10E946214FE01F5CF2091000172
:103BE00030E0A8EEB3E00E9470EBC60ED71EE81ED0
:103BF000F91EC092A302D092A402E092A502F09214
:103C0000A602DF91CF911F910F91FF90EF90DF906F
:103C1000CF9008950F931F93CF93DF9300D000D0E0
:103C2000CDB7DEB7809194048370833011F160E0EA
:103C30008FEA98E00E94D1B8E4EBF4E164918F013F
:103C40000F5F1F4F662331F088EB92E10E946214F0
:103C5000F801F4CFE0EAF8E064918F010F5F1F4FA5
:103C6000662309F43DC088EB92E10E946214F801DA
:103C7000F3CF1DD880E090E0A0E9B2E480939A04ED
:103C800090939B04A0939C04B0939D048091AE04F8
:103C90009091AF04A091B004B091B10480939E04C0
:103CA00090939F04A093A004B093A10480E090E0BF
:103CB000A0E7B2E48093960490939704A0939804AD
:103CC000B093990419821A821B821C82AE014F5F45
:103CD0005F4F6AE974E086E994E08FDB82E03EDDC5
:103CE0000F900F900F900F90DF91CF911F910F9138
:103CF0000895CF93DF93E2EAF7E06491EF01219614
:103D0000662331F088EB92E10E946214FE01F5CF48
:103D100087EB94E00E94075DE3E9F7E06491EF012F
:103D20002196662331F088EB92E10E946214FE0135
:103D3000F5CFDF91CF9108958091BA048823A9F03F
:103D400083E50E94D415882381F00E941716AB01E9
:103D5000BC01409325075093260760932707709373
:103D6000280784E796E00C9492500895CF93DF9350
:103D700083E40E948915882399F0E4E8F7E06491D0
:103D8000EF012196662331F088EB92E10E946214E4
:103D9000FE01F5CF87EB94E0DF91CF910C944D5D60
:103DA00087EB94E0DF91CF910C947B5E0F931F9390
:103DB000CF93DF93CDB7DEB769970FB6F894DEBF28
:103DC0000FBECDBF0E94F4A16E8B7F8B888F998F21
:103DD000BE016F5F7F4FCE0146960E94C91460E01E
:103DE000CE0101960E94AAB8E4EBF4E164918F0140
:103DF0000F5F1F4F662331F088EB92E10E9462143F
:103E0000F801F4CFBE016F5F7F4F87E797E00E9414
:103E100040936AE088EB92E10E94621469960FB6C3
:103E2000F894DEBF0FBECDBFDF91CF911F910F91F0
:103E30000895CF938091B90481110E94E783809106
:103E4000BA048823A9F180E50E94D415882321F0C3
:103E50000E944816C82F04C080E50E948915C82F0B
:103E60006091690970916A092C2F41E087EB94E019
:103E70000E94B46083E50E94D415882381F00E94DB
